:020000004C288A
:08000800F53081000608F03913
:10001000CB00C901CA010C3086006A206A206A2020
:100020006A200B30CE000608C500C51CCA0A451C54
:10003000C90ACE03031D13288601C90D49080319F7
:100040001430EB3E0318FF30CD00CA0D4A080319E7
:100050001430EB3E0318FF30CC00C60A031D3628CF
:10006000F030C6004C08C7004D08C800C70AC80ACF
:100070004708031D4028FF30C70085150515412896
:1000800085114808031D4928FF30C8000514851450
:100090004A2805100B11090083018316E030850002
:1000A000F33086000730810083121F308500F33063
:1000B0008600CB01F5308100FF30C700C800CC00BE
:1000C000CD008B168B17FA30CC00CD0066280800C7
:1000D00000000800FD30CF00CF0A031D6C2800008F
:0600E00071280000080079
:00000001FF
